:100000000C943B030C9458030C9458030C94580321
:100010000C9458030C9458030C9458030C945803F4
:100020000C9458030C9458030C946D120C94AF115B
:100030000C941F1A0C9458030C9458030C945803F6
:100040000C9458030C9458030C9458030C945803C4
:100050000C94E91C0C94D2190C9458030C9458037A
:100060000C9458030C9458030C9458030C945803A4
:100070000C9458030C9458030C9458030C94580394
:100080000C9458030C9458030C9458030C94580384
:100090000C9458030C9458030C9458030C94580374
:1000A0000C9458030C9458030C945803B604B804E9
:1000B0001105C004F804D0041E058205F6058A0562
:1000C000540558058E055B0591059C056605EC05F4
:1000D0006A05A0056E05A405CE057205A805D8051C
:1000E0007805AE05B8055F059505620598057D059F
:1000F000B305C405E405E60550058605FF0525069C
:100100002B0619061F06310637063D063607360749
:1001100068076807E70703080409040908087C085A
:100120008D088D08940C970CD20CEB0CF20CFD0C86
:10013000000D000D000DDE0DDE0D440D470D4B0DC5
:10014000710D940D970D9A0DBE0DBF0FE60F97110F
:10015000E60F97113210551097114B115B110000EB
:10016000000000000000000000000000000000008F
:10017000000000000000000000000000000000007F
:1001800000007E0F00D4FFFFFFC7000000780000D2
:100190000000000000002A2B2800000000000000E2
:1001A00000000000000000000029000000002C1EDC
:1001B0003420212224342627252E362D3738271E99
:1001C0001F202122232425263333362E37381F04BF
:1001D00005060708090A0B0C0D0E0F101112131457
:1001E00015161718191A1B1C1D2F3130232D350415
:1001F00005060708090A0B0C0D0E0F101112131437
:1002000015161718191A1B1C1D2F3130354C0501F6
:100210000902A10185020901A100050919012908A6
:100220001500250195087501810205010930093184
:100230001581257F95027508810609381581257F6E
:10024000950175088106050C0A38021581257F95F0
:100250000175088106C0C005010980A10185031947
:10026000012AB700150126B700950175108100C05D
:10027000050C0901A101850419012AA00215012616
:10028000A002950175108100C005010906A1018534
:1002900006050719E029E715002501950875018174
:1002A000020507190029EF1500250195F075018158
:1002B0000205081901290595057501910295017539
:1002C000039101C00660FF0961A1010962150026C2
:1002D000FF009520750881020963150026FF00952F
:1002E0002075089102C005010906A101050719E062
:1002F00029E715002501950875018102950175080A
:1003000081010507190029FF150026FF00950675D4
:1003100008810005081901290515002501950575B5
:10032000019102950175039101C009025B0003016F
:1003300000A0FA09040000010301010009211101D4
:10034000000122440007058103080001090401009F
:10035000020300000009211101000122220007050B
:1003600082032000010705030320000109040200A5
:10037000010300000009211101000122B600070558
:1003800084032000011201000200000008254068DB
:100390004D0101010200010A034D004600360038FC
:1003A0000000000C03640069003000690062000076
:1003B0000004030904000000000000000000000029
:1003C00001010203040506080A0C0F1114181C2071
:1003D00024292E33393F464C535B626A7179818AF6
:1003E000929AA2AAB2B9C1C8CFD5DCE1E7EBF0F48A
:1003F000F7FAFCFDFEFFFEFDFCFAF7F4F0EBE7E197
:10040000DCD5CFC8C1B9B2AAA29A928A8179716AA1
:10041000625B534C463F39332E2924201C1814119B
:100420000F0C0A0806050403020101000000000089
:10043000000000000029001E001F002000210022F3
:1004400000230024002500260027002D002E002A6E
:100450000049004B002B0014001A0008001500177B
:10046000001C0018000C00120013002F0030003197
:10047000004C004E00390004001600070009000A75
:10048000000B000D000E000F00330034002800E1C7
:10049000001D001B000600190005001100100036A9
:1004A0000037003800E5005200E000E300E2002CD5
:1004B000002152E600E400500051004F000000000F
:1004C000000000000035003A003B003C003D003ECB
:1004D000003F004000410042004300440045002A24
:1004E00000A9004A000100010001005200010001C2
:1004F0000001000100010001000100010005780178
:1005000000AA004D0001000100500051004F000101
:1005100000010001000100010001000100010001D3
:1005200000010001000100010001000100A800011C
:1005300000010001000100A800010001000100010C
:1005400000010001000100AC00AE00AB00000000A3
:100550000000000000010001000100010001000195
:100560000001000100010001000100010001000183
:100570000001000100010001000100010001000173
:100580000001000100010001000100010001000163
:100590000001000100010001000100010001000153
:1005A0000001000100010001000100010001000143
:1005B0000001000100010001000100010001000133
:1005C0000001000100010001000100010001000123
:1005D0000001000100010001000100010000000015
:1005E0000000000000010001000100010001000105
:1005F00000010001000100010001000100010001F3
:1006000000010001000100010001000100010001E2
:1006100000010001000100010001000100010001D2
:1006200000010001000100010001000100010001C2
:1006300000010001000100010001000100010001B2
:1006400000010001000100010001000100010001A2
:100650000001000100010001000100010001000192
:100660000001000100010001000100010000000084
:1006700000000000000011241FBECFEFDAE0DEBF53
:10068000CDBF11E0A0E0B1E0E0E6F7E402C00590E4
:100690000D92A836B107D9F722E0A8E6B1E001C073
:1006A0001D92AB38B207E1F70E9448090C94AE23C3
:1006B0000C940000A8E0B0E0E0E6F3E00C946A23BC
:1006C000FC018481882309F4DFC57F0121E040819A
:1006D00051816281738195810E94B7208C01F7015D
:1006E0008581882309F4B4C1980137572038310532
:1006F00008F032C1003108F0DDC28FEF93E00E94B4
:1007000097228111D7C238E6A32E32E0B32E002300
:1007100079F0A114F4E0BF0609F4CCC2C5010E942F
:100720009722811101C001502FEFA21AB20AEFCF18
:10073000CE0101962C0188E0F20111928A95E9F729
:100740002AE0322E85010F5F1F4FC5010E949722BC
:1007500089831A82882309F4ADC2813009F041C02F
:100760006501F2E0CF0ED11CC8010E9497228A8356
:10077000882309F49FC29FEF980F933060F423E021
:10078000A20EB11CC6010E9497228B83882309F414
:1007900091C21C8229C0843031F54E0133E0830EB2
:1007A000911C02E010E056018FEFA81AB80AC601AA
:1007B0000E949722F40181934F01882309F47AC2A1
:1007C0008C3741F4E2E0F0E0EC0FFD1FE00FF11F89
:1007D00010820AC00F5F1F4F65010730110519F71E
:1007E00069C2580101C056018201F801208122230B
:1007F00009F4A8CF213009F053C08181813081F400
:100800006801F2E0CF0ED11CF8018281893319F41E
:1008100060E570E002C060E070E00E949F2015C0BB
:10082000823049F46801F2E0CF0ED11CF8018281D8
:100830000E94E81F0AC0833051F46801F2E0CF0E35
:10084000D11CF80182810E948E1F860182C08430F3
:1008500019F00F5F1F4F7DC0F80122810E5F1F4FFF
:1008600080E090E030E0205331092A30310568F40F
:10087000389EA001399E500D1124C901840F951F87
:100880000F5F1F4FF8012081EDCF009709F461C081
:10089000EFE9FFE03197F1F700C000000197F5CFD5
:1008A000E22FF0E0E257FE4F2490822F8695869546
:1008B000869590E0FC01E258FE4F64902770712C01
:1008C000022E02C0759467940A94E2F7F1E06F2259
:1008D0007724FC01E259FE4F8490912C022E02C035
:1008E000959487940A94E2F731E083229924FC01DD
:1008F000E25AFE4FC490D12C02C0D594C7942A95D9
:10090000E2F781E0C822DD246114710419F081EE60
:100910000E94E81F8114910419F086EE0E94E81FDE
:1009200060E070E0822D0E949F208114910419F0F4
:1009300086EE0E948E1F6114710419F081EE0E94F0
:100940008E1FC114D10429F060E070E08CE20E9497
:100950009F200F5F1F4F49CFF801F857E730F1058F
:1009600008F076C0EA5AFF4F0C94432383E001C09D
:1009700080E00E94312280914F020E9400229AC1A1
:1009800080914F02982F96959695969549F1915E94
:10099000990F990F990F8770892B80934F0214C07C
:1009A00090914F02892F8695869586958F5F8F71DE
:1009B0009770843008F03FC0880F880F880F892B0C
:1009C00080934F0280914F02887F91E009F490E07C
:1009D00080914F0290FB80F980934F020E94002289
:1009E00080914F028695869586950E94621D62C110
:1009F00020914F02822F869586958695482F50E04C
:100A00004330510554F48F5F982F990F990F990F28
:100A1000822F8770892B80934F0280914F028160D3
:100A2000DBCF80914F0280FF03C00E944B2242C166
:100A30000E9458223FC190934F02C4CF80914F0231
:100A400081FF03C00E94062235C10E941C2232C1D0
:100A5000F801E851FC47E730F10508F4E6C08823C7
:100A600009F43CC1109262029801305723323105DB
:100A700008F00CC184E090E00E949F2290936A02EB
:100A800080936902F801E150F047E232F10520F469
:100A9000E35AFF4F0C944323809169028160ACC0FC
:100AA00080916A028860B4C0809169028260A4C0AB
:100AB0008091690220C08091690288609DC0809108
:100AC0006A021EC080916A028260A2C0809169029F
:100AD000806192C08091690280628EC080916902BB
:100AE00080648AC00E94741E80916902806884C0FC
:100AF00080916902886084607FC080916A02826010
:100B0000816086C0809169028E7F76C080916A0282
:100B1000877F7EC0809169028D7F6EC0809169025F
:100B200020C080916902877F67C080916A021EC0E1
:100B300080916A028D7F6CC0809169028F7E5CC05B
:100B4000809169028F7D58C0809169028F7B54C06B
:100B50000E94741E809169028F774EC08091690255
:100B6000877F8B7F49C080916A028D7F8E7F50C0C6
:100B70008091690282FB222720F991E0922790FB65
:100B800082F990FB83F938C080916A02982F909582
:100B900091708E7F892B90FB81F93AC08091690218
:100BA00086FB222720F991E0922790FB86F924C04A
:100BB0000E94741E8091690287FB222720F991E030
:100BC000922790FB87F918C061E001C060E08EE0D9
:100BD00090E00E94B5221EC08091690284FB22270A
:100BE00020F991E0922790FB84F906C08091690278
:100BF000982F909590FB80F9809369020BC08091AB
:100C00006A0283FB222720F991E0922790FB83F967
:100C100080936A026091690270916A0284E090E0B8
:100C20000E94D3220E94741E45C0E158FF4F0C94CD
:100C3000432306E221EE41EE6AE17CE723C007E2AE
:100C400025EE45EE6BE17CE71DC006E221EE40EEAD
:100C500068E17CE717C007E225EE44EE69E17CE736
:100C600011C006E221EE42EE6CE17CE70BC007E228
:100C700025EE46EE6DE17CE705C008E221E045EE99
:100C80006EE17CE7C7010E94411B14C00631FCE7FE
:100C90001F0709F0E1C2809121028A7A91E009F4EC
:100CA00090E090936A01811117C089E20E94761A40
:100CB0000E94D9168091F601877009F4E5C2F70108
:100CC0008581882309F4E0C280916A0282FFDCC238
:100CD00082E00E942B17D8C285E3E8CF06312CE7CB
:100CE000120751F480916A01811104C089E20E94C7
:100CF000481ADECF85E3FBCF07373CE7130711F433
:100D000081E0BAC208379CE7190709F4B4C2980118
:100D1000205E324520323105A8F4811115C00F71D3
:100D200081E090E0FC0102C0EE0FFF1F0A95E2F7A0
:100D30008F016E2F83E090E00E94B522802F0E94E9
:100D40004E1EB8CF8823E9F10330FCE71F0729F1D5
:100D500048F401153CE7130791F001308CE71807C0
:100D600011F12FC00B359CE7190741F10C35ECE769
:100D70001E07E1F00A351C4721F581E020C00E94E2
:100D8000741E2FEF34E38CE0215030408040E1F7B7
:100D900000C000000E94C1198DCF6FEF7FEF80E08F
:100DA00090E00E94D3220E946C2184CF80916A023D
:100DB00082FB882780F991E0892701C080E00E94AA
:100DC0004217F701858100811181882349F0C8010C
:100DD0000E948D1DD82E682FC8010E94FD1D04C0E1
:100DE000C8010E94C91DD82EB8018D2D0E948315FF
:100DF0000E9491158C01A82EF701B58096809294DF
:100E00009FE099228091F601877001F1BB20F1F0FB
:100E1000812F807F803469F080E2800F8830B0F0CD
:100E2000812F807E803229F4F1E0F01778F4992048
:100E300069F080916A0282FF09C082E00E942B174C
:100E40008091F6018770DD24D3948111D12CC12EBD
:100E5000C2948FE0C8228C2D90E08C30910508F070
:100E6000D3C1FC01EA57FF4F0C944323812F807FAD
:100E70001F70882311F01295107FBB20B9F0112349
:100E800009F4B0C180E2800F883010F0A11006C0D4
:100E900090912102192B1093210205C09091F80125
:100EA000192B1093F8010E94D9169CC1802F0E9423
:100EB0008E1F112309F4A8C1005E083080F1AA201A
:100EC00071F110959091F80119231093F8012AC03F
:100ED000812F807F1F70803211F01295107FAA2021
:100EE00029F021E0A21609F44DC058C080916A0291
:100EF00082FD1BC0BB2069F0112339F03091210223
:100F0000312B309321020E94D91680E00E94E81F05
:100F10007BC180E00E948E1F112309F475C1812FCF
:100F20000E94D2160E94D9166FC1BB2081F0992071
:100F3000C9F131E0931268C13091F701812F832309
:100F4000181709F461C1312B3093F7015DC191107D
:100F50005BC1812F0E94A51E3091F701812F832351
:100F600029F0812F809538233093F70120916B0170
:100F7000812F822309F448C1312F309523232093F8
:100F80006B0142C1BB2029F085E0891508F43CC102
:100F900009C094E0991508F437C115C0BB2031F0A1
:100FA000911020C1812F0E94AC1E2EC1992059F0B2
:100FB000093309F026C1EFEFF7EE23E0E150F040EE
:100FC0002040E1F71CC1812F0E94A51E1DC1812F69
:100FD00086958695837019F0813059F015C1BB2034
:100FE00019F0C801937002C080E090E00E94D21A0C
:100FF00011C1BB2019F0C801937002C080E090E0DD
:101000000E94AD1A07C16B2D802F0E94B61E02C12F
:10101000812F8370A9F5B110FBC0402F42954695F2
:101020004770440F440F802F8F7090E09C01042E76
:1010300001C0220F0A94EAF704FF08C08FE090E095
:1010400001C0880F4A95EAF7809501C080E01695A7
:1010500016951370123069F088F490917C0111306C
:1010600019F0822B892302C0922B892B0E944E1EDD
:10107000CFC0822B90917C018927F8CF822BF6CFAD
:10108000BB2019F0812F817001C08695882309F457
:10109000BFC0402F429546954770440F440F802FA4
:1010A0008F7090E09C01042E01C0220F0A94EAF791
:1010B00004FF08C08FE090E001C0880F4A95EAF76E
:1010C000809501C080E0169516951370123059F086
:1010D00078F490917D01113019F0822B892309C099
:1010E000922B892B06C0822B90917D01892701C00C
:1010F000822B0E94321E8CC01F70BB2039F0812FC2
:101100000E94421E802F0E94AC1E82C0802F0E942F
:10111000A51E812F0E94351E7BC0802F32EFA316A3
:1011200081F13A1538F090EFA91659F0E1EFAE16BB
:1011300019F154C0F3EFAF1659F124EFA216C1F024
:101140004DC0BB2081F034E0391508F45DC01F713B
:1011500081E090E0012E01C0880F0A94EAF7909197
:101160007D01892720C085E0891508F44DC0EFCFA7
:1011700080916A0282FD1AC0BB2029F0812F8F71F5
:1011800020C0BB20D9F3812F8F710E94351E3CC037
:10119000BB2041F01F7181E0012E01C0880F0A942D
:1011A000EAF701C080E00E94321E2EC0BB2061F031
:1011B000812F8F7198E0899F9001112423602093E3
:1011C000F6010E94421E20C081E00E942B17E1E040
:1011D000E915D0F482E00E942B1716C0BB2021F045
:1011E000992061F2802F92CE992069F2893349F4D7
:1011F000FFEF27EE33E0F15020403040E1F700C030
:101200000000802F0E948E1F88EF8C0D843010F418
:101210000E94F71ADD20A9F08091F60180FD11C02F
:10122000F70115828695869586950E94421EC70114
:101230000E945A038091F6018695869586950E94B4
:10124000351E20E0F70140815181628173818481E4
:1012500095810E94B72018C00737ECE71E0711F4EC
:1012600081E006C00837FCE71F0709F050CD82E097
:101270000E94421E03C082E00E94351E43E062E0ED
:1012800081E00E94431916CD2896E2E10C94862352
:10129000A6E2B0E0EEE4F9E00C946A2385B780683A
:1012A00085BF85B7806885BF84B7877F84BF0FB649
:1012B000F894A895809160008861809360001092F6
:1012C00060000FBE90E080E80FB6F8948093610054
:1012D000909361000FBE81E080930D0186E893E159
:1012E00090936901809368010E94F3110E94121289
:1012F0008091E20084608093E20078948091AB0159
:101300008823A1F01091E9001F709091EC00892FC3
:10131000817090FD80E8182B1092E9008091E80020
:1013200083FD0E94D70E1F701093E90082E084BDF8
:1013300093E095BD9AEF97BD80936E000E94281BA5
:10134000811102C00E94AB1C0FE011E087E1E82E82
:1013500081E0F82ED8018D918D018F3F11F00E9410
:10136000B914E016F106B1F707E111E0B0E2EB2E97
:10137000B1E0FB2EF80181918F018F3F11F00E94A7
:10138000B914E016F106B1F780E1E0E9F1E0DF0120
:10139000282F1D922A95E9F7ECE6F1E0DF011D9276
:1013A0008A95E9F780E090E00E949F22853E9E4F5B
:1013B00021F40E94281B811163C065EE7EEF80E05E
:1013C00090E00E94D32260E082E090E00E94B5228B
:1013D00081E080937C0161E083E090E00E94B5228F
:1013E00060E074E184E090E00E94D32260E086E057
:1013F00090E00E94B52260E087E090E00E94B52274
:1014000040E050E0BA0188E090E00E94C72260E02E
:1014100083E290E00E94B52260E08CE090E00E94C0
:10142000B52260E08DE090E00E94B52219821A8218
:101430001B821C821D821E821F82188648E050E09B
:1014400067E170E0CE0101960E94A52240E050E0E5
:10145000BA018FE190E00E94C72280E00E94091B40
:101460000E94AB1C40E050E0BA018FE090E00E9487
:10147000C72240E050E0BA0183E190E00E94C72219
:1014800082E090E00E94972280937E0184E090E0C9
:101490000E949F2290936A02809369020E94D01456
:1014A000EFEFF6E721E0E150F0402040E1F700C027
:1014B00000000E94D0148091900180FF08C06FEF5F
:1014C0007FEF80E090E00E94D3220E94C11983E068
:1014D00090E00E9497220E944E1E259A2D9882E845
:1014E0008093800089E1809381008FEF9FEF90933C
:1014F0008700809386000E94702280914F0281FFB6
:101500000BC0109252021092510210925002809120
:101510006F00816080936F000E94702280E091E0F4
:101520009093660280936502552453942224239459
:101530008E010F5F1F4F8091AB01853009F046C0CF
:10154000A0E4FA2E8091AB01853009F039C080917A
:10155000AB01843031F180E00E94312210926B02A5
:1015600088E190E00FB6F894A895809360000FBED4
:10157000F092600083B7817F846083BF83B781600E
:1015800083BF7894889583B78E7F83BF0FB6F89416
:10159000A89580916000886180936000109260003F
:1015A0000FBE0E94D014E0E9F1E081919191892B66
:1015B00009F00DC3A0EAB1E0AE17BF07B1F7C2CF83
:1015C0000E94741E0E9470220E94F71A0E94D0147A
:1015D000EFE7EE2EE1E0FE2EF0E96F2EF1E07F2E38
:1015E000D301F701219131918D919D91822793270C
:1015F00021E0EF38F20719F0892BA1F305C0892B00
:1016000019F40E94AE163EC0412CD3018D909D90DE
:101610003D01F701A080B180A824B924A114B10430
:1016200041F1312CCC24C394D12CC6018A219B21B9
:10163000892BB1F039A24AA20E94131A9CA38BA352
:101640002DA291E0960128213921232B09F490E065
:101650009EA349A15AA16BA17CA18DA10E94DC206F
:101660003394CC0CDD1CF9E03F12DFCFD7018D9213
:101670009C924394B2E0EB0EF11CE8E04E12C5CF11
:101680000E94071A86E0EAE5F2E0D80101900D9287
:101690008A95E1F7B0905B02D0905C02F0905D0219
:1016A000E0905E02C0905F0210925C0210925D02B8
:1016B00010925E0210925F02D11003C0FF2009F465
:1016C0004BC080915802909159020E94F8199C01D8
:1016D00090915302992309F4A0C225313105E0F11C
:1016E0009F3F19F09F5F90935302DD2061F00E94AD
:1016F000111C1D1414F491E001C09FEF899F802DEF
:10170000112480935C02FF2061F00E94111C1F14C1
:1017100014F09FEF01C091E0899F802D11248093E8
:101720005D0280915C028823B9F0A0905D02AA203E
:1017300099F00E94311C882319F080935C0202C04A
:1017400050925C028A2D0E94311C882319F08093EC
:101750005D0202C050925D02E11003C0CC2009F48A
:101760004BC080915602909157020E94F8199C013B
:1017700090915402992309F455C221353105E0F1C5
:101780009F3F19F09F5F90935402EE2061F00E94FA
:10179000EF1B1E1414F491E001C09FEF899F802D70
:1017A000112480935E02CC2061F00E94EF1B1C1478
:1017B00014F09FEF01C091E0899F802D1124809348
:1017C0005F0280915E028823B9F0A0905F02AA2098
:1017D00099F00E94311C882319F080935E0202C0A8
:1017E00050925E028A2D0E94311C882319F080934A
:1017F0005F0202C050925F0280915B028B111AC09F
:1018000080915C02882311F08D1114C080915D02DB
:10181000882311F0F8120EC080915F02882311F026
:101820008C1108C090915E02992331F081E0E91299
:1018300004C002C081E001C080E080FD15C080913D
:101840005C0281110FC080915D0281110BC08091FB
:101850005E02811107C081E090915F02911103C087
:1018600080E001C081E080FD0E94C51BBA82DB825E
:10187000FC82ED82CE8286E0F801AAE5B2E001901A
:101880000D928A95E1F70E94F71A90918F018917BE
:1018900021F080938F010E94071A8091AB01843060
:1018A00009F049CE83E08093E9008091E80082FF4F
:1018B00042CE8091E80085FF21C00E945313811120
:1018C0001BC050E2C52ED12C780109C08091F100D7
:1018D000D7018D937D01B1E0CB1AD10869F08091D9
:1018E000E80085FDF3CF8091E8008B778093E800D6
:1018F0000E945313882399F391E001C090E08091F6
:10190000E8008B778093E800992309F414CE2981AD
:10191000822F90E0FC013197E331F10508F04EC1D0
:10192000EE56FF4F0C9443231A828CE0B2C08A819A
:10193000823009F469C150F4813009F03FC10E943E
:10194000071A9B838C837D836E833AC1833041F079
:10195000843009F033C11B821C821D821E8230C17B
:101960006B81D80180E090E0262F30E0A901480F7C
:10197000591F4830510508F023C1E62FE80FF0E069
:10198000EE0FFF1FE057FE4F4081518113965C938D
:10199000139714964C931497019612968E309105D6
:1019A00029F70EC18A81823019F0853051F006C1C5
:1019B0006B817C818D819E810E9449230E94041B42
:1019C000FFC080914F0280FF03C00E944B22F8C0ED
:1019D0000E945822F5C04C816B818A810E94BB1CF9
:1019E0009D8319C12D813E813227232732274C81C7
:1019F0006B818A810E944F1CE3C00E94761CE0C06C
:101A00008A81813009F0DAC02830F1F02930B9F14B
:101A10008B81813019F0823071F0D2C08C81E3E08B
:101A20008E9FC00111246FEF70E00E94F922862F73
:101A30000E943122C5C08C81811103C00E94062200
:101A4000BFC00E941C22BCC08B81813049F0823013
:101A500009F0B6C080914F02869581708C83B0C02A
:101A600080914F02869586958695FFEF8F9FC001E6
:101A7000112463E070E00E94F9226C83A1C0809180
:101A80004F020E9400229CC020E12A8399C05A8202
:101A900088E98B8395C0EA80FB80FE24EF24FE2436
:101AA000CC80D12C5801C70188599D4F9501201B2E
:101AB000310B2C153D0508F083C0A8E9EA16A1E01A
:101AC000FA0628F40E949722F501848303C0D50109
:101AD00014961C92BFEFEB1AFB0AEFEFAE1ABE0A88
:101AE000E2CFEA80FB80FE24EF24FE24CC80D12CC0
:101AF0005801C70188599D4F9501201B310B2C15AA
:101B00003D0508F05DC0F8E9EF16F1E0FF0628F4A6
:101B1000D50114966C910E94B522BFEFEB1AFB0A17
:101B2000EFEFAE1ABE0AE5CF0E943F1C49C084E029
:101B30008A8346C0EA80FB80FE24EF24FE24CC800A
:101B4000D12C5801C70188969501201B310B2C150B
:101B50003D05B0F5F0E4EF16F2E0FF0630F40E9428
:101B60009722D50114968C9302C0F5011482FFEFE1
:101B7000EF1AFF0A2FEFA21AB20AE4CFEA80FB8025
:101B8000FE24EF24FE24CC80D12C5801C701889676
:101B90009501201B310B2C153D0590F4A0E4EA16AD
:101BA000A2E0FA0620F4F50164810E94B522FFEF5D
:101BB000EF1AFF0A2FEFA21AB20AE8CF8FEF89833C
:101BC00040E250E0B80182E00E946819B4CC8091F4
:101BD000AA01882309F4B6CCB0E1B9BDE2E1E9BDC0
:101BE00009B400FEFDCF8091D8008F7D8093D8008E
:101BF0008091E00082608093E0008091E00081FDB0
:101C0000FCCF0E94741E9ECC87E290E00E94972237
:101C10001B821C821D828E83D3CF2B30310508F0AE
:101C200061CD9ACD2B30310508F0ACCDE5CD80915A
:101C3000AD0187FF11C08091E80082FD05C0809151
:101C4000AB018111F8CF11C08091E8008B770BC0F8
:101C50008091AB01882349F08091E80080FFF8CFA4
:101C60008091E8008E778093E8000895982F973050
:101C700068F59093E900981739F07091EC00209185
:101C8000ED005091F00003C0242F762F50E021FD8D
:101C900002C09F5FECCF3091EB003E7F3093EB00B2
:101CA0003091ED003D7F3093ED003091EB003160DD
:101CB0003093EB007093EC002093ED005093F00014
:101CC0002091EE0027FDE5CF80E008958F7080938E
:101CD000E90081E008952091B3013091B401261705
:101CE000370748F06115710539F42091E8002E7727
:101CF0002093E80001C0B901FC0120E061157105E5
:101D000079F18091AB018823F1F18530F1F1809177
:101D1000E80083FD3CC08091E80082FD2EC08091E8
:101D2000E80080FFEBCF2091F3008091F20090E07B
:101D3000922B6115710551F08830910538F421918D
:101D40002093F100615071090196F3CF21E00897CB
:101D500009F020E08091E8008E778093E800CECFF4
:101D60002111CFCF0AC08091AB01882361F085306B
:101D700061F08091E80083FD0AC08091E80082FF55
:101D8000F2CF80E0089582E0089583E0089581E035
:101D9000089543E050E0BC0184E00E946819089572
:101DA00046E050E0BC0184E00E9468190895AAE270
:101DB000B0E0EDEDFEE00C947923EDEAF1E085EB87
:101DC00091E02091F10021938E179F07D1F7809128
:101DD000AE01833009F463C030F4813071F0823099
:101DE00009F4A2C0B9C08A3009F48EC08B3009F45E
:101DF0006EC0893009F0B0C020C08091AD01813A39
:101E000009F0AAC08091E800877F8093E800809164
:101E1000B1019091B201892B21F468E081EA91E04F
:101E200003C060E080E090E070E00E946B0E809163
:101E3000E8008B778093E8008FC08091AD018132FC
:101E400009F08AC08091B1019091B201009719F018
:101E5000029709F081C08091E800877F8093E800B5
:101E60008091E80082FD05C08091AB018111F8CF1F
:101E700073C02091F3008091F20090E0922B0297C2
:101E800031F48091F100813011F0863021F480919D
:101E9000F10080930B018091E8008B7759C080910D
:101EA000AD01813A09F058C08091B1019091B20121
:101EB000892B09F051C08091E800877F8093E8006A
:101EC0008091E80080FFFCCF80910C013CC08091A4
:101ED000AD01813209F040C08091B1019091B20111
:101EE000892BD1F58091E800877F8093E8000E94DC
:101EF000170E81E09091AF01911101C080E08093B5
:101F00000C010E94741E28C08091AD01813221F520
:101F10008091E800877F8093E8000E94170E8091EF
:101F2000B00180930A0118C08091AD01813AA1F4FB
:101F30008091E800877F8093E8008091E80080FF2F
:101F4000FCCF80910A018093F1008091E8008E77A8
:101F50008093E8000E94170E8091E80083FFE7C19C
:101F60008091AD019091AE01492F50E04A3051056A
:101F700008F0DDC1FA01EB55FF4F0C944323803884
:101F800021F0823809F0D3C108C08091A901909155
:101F9000AA01992389F082600FC08091B1018F70EE
:101FA000873008F0C4C18093E9008091EB0085FB85
:101FB000882780F91092E9009091E800977F90932C
:101FC000E8008093F1001092F10071C1282F2D7F5D
:101FD00009F0ADC1882319F0823061F0A8C1809169
:101FE000AF01813009F0A3C1933009F080E0809304
:101FF000AA012EC08091AF0181112AC08091B10148
:102000008F702FEF280F263008F091C18093E900E0
:102010002091EB0020FF1CC0933021F48091EB0055
:10202000806214C09091EB0090619093EB0021E0EE
:1020300030E0A90102C0440F551F8A95E2F7409392
:10204000EA001092EA008091EB0088608093EB0038
:102050001092E9008091E800877F8093E8000E9459
:10206000170E65C1811163C11091AF011F77809177
:10207000E3008078812B8093E3008091E800877FE4
:102080008093E8000E94170E8091E80080FFFCCF4B
:102090008091E30080688093E300111102C082E028
:1020A00001C083E08093AB0142C18058823008F0C8
:1020B0003EC12091AF013091B0012C3D53E0350776
:1020C00079F583E08A838AE289834FB7F894DE0149
:1020D000139620E03EE051E2E32FF0E050935700EA
:1020E000E49120FF03C0E295EF703F5FEF708E2F09
:1020F00090E0EA3010F0C79601C0C0968D939D9392
:102100002F5F243149F74FBF8091E800877F80938C
:10211000E8006AE270E0CE0101960E946B0EB5C045
:102120008091B1019091B201432F55274330510561
:10213000A9F068F44130510509F408C14230510555
:1021400009F0F5C08BE590E0EAE2F3E04BC04132E4
:10215000510529F14232510589F1E9C0C901992798
:1021600081309105A1F058F0029709F0E0C0E7E94D
:10217000F3E0E4918E2F90E0E7E9F3E030C0E1EB8B
:10218000F3E0E4918E2F90E0E1EBF3E028C0E3EA86
:10219000F3E0E4918E2F90E0E3EAF3E020C0833097
:1021A000910508F0C4C0880F991FFC01E75DFE4F40
:1021B0000190F081E02D89E090E014C0833091051A
:1021C00008F0B5C0FC01EE0FFF1FED5DFE4F019062
:1021D000F081E02DDC01A05EBE4F8C9190E0009775
:1021E00009F4A5C02091E800277F2093E800209102
:1021F000B3013091B4018217930708F49C0140E0C9
:102200002115310589F18091AB01882309F43DC086
:102210008530D9F18091E80083FD37C08091E800D6
:1022200082FD2FC08091E80080FFEACF4091F3004B
:102230008091F20090E0942B2115310559F08830FF
:10224000910540F444914093F100319621503109B9
:102250000196F2CF41E0089709F040E08091E80054
:102260008E778093E800CCCF4111CDCF0AC080910A
:10227000AB01882351F0853041F08091E80083FD67
:1022800004C08091E80082FFF2CF8091E8008B7754
:102290008093E8004CC0803809F049C08091E80084
:1022A000877F8093E8008091AC018093F10080915A
:1022B000E8008E77D2CE81113AC08091AF01909123
:1022C000B001992702979CF58091E800877F809361
:1022D000E8001091AF011093AC010E94170E11118C
:1022E00006C08091E30087FD02C081E001C084E068
:1022F0008093AB0142E061EC81E00E94360E42E245
:1023000061EC84E00E94360E42E261EC82E00E94C1
:10231000360E42E260EC83E00E94360E8091AB0103
:10232000843011F081E001C082E080930D01809142
:10233000E80083FF10C08091E800877F8093E80069
:102340008091EB0080628093EB0005C082E190E019
:10235000E5E8F3E047CFAA96E3E00C9495231F92BB
:102360000F920FB60F9211242F933F934F935F93C9
:102370006F937F938F939F93AF93BF93CF93DF938D
:10238000EF93FF93C091E900CF708091EC00D82FBC
:10239000D17080FDD0E81092E9008091F000877F35
:1023A0008093F00078940E94D70E1092E9008091FB
:1023B000F00088608093F000CD2BCF70C093E900CF
:1023C000FF91EF91DF91CF91BF91AF919F918F914D
:1023D0007F916F915F914F913F912F910F900FBE21
:1023E0000F901F901895E8EDF0E080818E7F80833C
:1023F0001092E2001092DA001092E100A0EEB0E03C
:102400008C9181608C9380818F77808319BCA7ED3C
:10241000B0E08C918E7F8C9380818F7E8083109230
:10242000A0010895A0E0B0E0E8E1F2E10C9474238B
:10243000C8EDD0E088818F7E8883E7EDF0E0808171
:102440008160808384E082BF81E08093A0018881E5
:102450008E7F888302EE10E0F80110821092DA007D
:1024600081EEC82ED12CF601108288818F77888367
:1024700088818068888388818F7D888319BC1092C9
:10248000AB011092AC011092AA011092A90190EE3A
:10249000E92EF12CF70180818B7F80838881816018
:1024A000888342E060E080E00E94360EF601808181
:1024B0008E7F8083F8018081816080838081886045
:1024C0008083F70180818E7F80838881806188830B
:1024D000CDB7DEB7E8E00C9490231F920F920FB6B1
:1024E0000F9211242F933F934F935F936F937F939A
:1024F0008F939F93AF93BF93EF93FF938091E100EE
:1025000082FF09C08091E20082FF05C08091E10056
:102510008B7F8093E1008091DA0080FF2AC0809158
:10252000D80080FF26C08091DA008E7F8093DA0089
:102530008091D90080FF18C080E189BD82E189BD0A
:1025400009B400FEFDCF81E08093AB018091A00132
:1025500081110FC00E94F3110E9412128091E200BB
:1025600084608093E20005C019BC1092AB01109208
:10257000A0018091E10080FF1AC08091E20080FFFD
:1025800016C08091E2008E7F8093E2008091E2008D
:1025900080618093E2008091D80080628093D800AF
:1025A00019BC85E08093AB0183E080930D0180919D
:1025B000E10084FF37C08091E20084FF33C080E1F6
:1025C00089BD82E189BD09B400FEFDCF8091D800AC
:1025D0008F7D8093D8008091E1008F7E8093E10011
:1025E0008091E2008F7E8093E2008091E200816022
:1025F0008093E2008091AC01882311F084E007C051
:102600008091E30087FD02C081E001C083E08093F8
:10261000AB018091AB01843011F081E001C082E018
:1026200080930D018091E10083FF2CC08091E20036
:1026300083FF28C08091E100877F8093E10082E0E2
:102640008093AB011092AC018091E1008E7F80936A
:10265000E1008091E2008E7F8093E2008091E200B1
:1026600080618093E20042E060E080E00E94360EEC
:102670008091F00088608093F00081E080930D01EC
:1026800080930C01FF91EF91BF91AF919F918F913A
:102690007F916F915F914F913F912F910F900FBE5E
:1026A0000F901F9018952091E4003091E50095E679
:1026B0004091EC00842F817040FF23C08091E8009E
:1026C00080FD1DC08091AB01882399F0853099F081
:1026D0008091EB0085FD11C04091E4005091E50030
:1026E0002417350729F3915011F09A01E1CF84E0C6
:1026F000089582E0089583E0089581E0089580E0E0
:1027000008954091E80042FFDDCF089580E00895EC
:102710009091690292FF10C041E0282F247124306B
:1027200009F040E031E0282F2871283009F030E02E
:10273000431711F02CE0822793FF10C041E0282FAF
:102740002471243109F040E031E0282F287128312C
:1027500009F030E0431711F02CE0822730916A0233
:1027600030FF10C051E0282F2171213009F050E0D6
:1027700041E0282F2871283009F040E0541711F06B
:1027800029E0822731FF10C041E0282F217121313B
:1027900009F040E031E0282F2871283109F030E0BD
:1027A000431711F029E0822794FD877E089582382F
:1027B000910569F1B0F48133910509F475C048F4CD
:1027C0008932910509F467C08A32910509F471C014
:1027D00008958533910509F459C089339105B9F0FD
:1027E0000895833E910589F138F4803E9105D1F03A
:1027F000823E910529F10895863E9105C9F1873EF3
:102800009105D9F1843E910509F06CC027C0209153
:10281000690220FD57C021FD55C020916A0223FDA9
:102820005BC008958091690280FD48C080916A0272
:1028300080FF48C08091690284FD46C083EE51C08C
:102840008091690282FF3CC0F5CF8091690282FDD0
:1028500037C080916A0280FD35C0ECCF80916A025A
:1028600081FF36C08091690284FD2EC087EE39C099
:102870008091690283FF2AC0F5CF8091690283FDB0
:1028800025C080916A0281FD23C0ECCF809169024E
:1028900085FD22C01FC08091690285FD1BC080910B
:1028A0006A0283FF19C00AC08091690286FD16C0C2
:1028B00017C08091690286FD13C010C089E311C062
:1028C00082EE0FC080EE0DC080E00BC086EE09C026
:1028D00084EE07C085E305C089E203C08AE201C037
:1028E00081E390E00895909121028091F801892B75
:1028F0009091F7019923E1F0892B90910C0191308F
:1029000041F49091690297FF04C09EE121E332E017
:1029100003C096E029E232E0F90120E0915028F06E
:1029200031913323D9F32F5FF9CF21111092F701A1
:1029300008952091F5019091BC0157E02917A9F065
:1029400030E0529FF001539FF00D1124E354FE4FED
:102950007181761306C07081781303C0758174137A
:1029600006C02F5F3F4F2770E9CF80E0089581E0D8
:102970000895F894E82FE295EF70F0E031A1282F48
:102980002F7081E090E001C0880F2A95EAF7982F18
:102990009095932391A392A1892B82A37894089573
:1029A000A0E1B0E0E6EDF4E10C946E23AE014F5FE0
:1029B0005F4F7A0180E1FA0111928A95E9F70FE001
:1029C00011E06A0197E1692E91E0792E88248394C1
:1029D000912CF80180818F3F09F447C0F894E82FCB
:1029E000E295EF70F0E021A18F70A40102C0440FC6
:1029F000551F8A95E2F7CA01922F982B91A392A1B5
:102A00008095892382A3789400C0E7E1F1E021E07A
:102A100030E0A12CB12C41914F3F89F0A42FA29519
:102A2000AF70B0E090968C9190E04F7002C0959599
:102A300087954A95E2F780FD02C0C90102C080E097
:102A400090E0A82AB92A220F331F51E0E032F5079F
:102A500011F7F80180818F3F11F00E94B914F0EA5C
:102A6000FA95F1F7F601B182A0820F5F1F4FF2E0F5
:102A7000CF0ED11C6016710609F0ABCF40E150E0DB
:102A8000B7018CE691E00E94A123892B91F080E1AF
:102A9000F701ACE6B1E001900D928A95E1F781E093
:102AA000809326020E94131A909325028093240299
:102AB0000CC080912602882341F0809124029091DD
:102AC00025020E94F819059710F480E018C040E133
:102AD00050E06CE671E080E991E00E94A123892B2F
:102AE00059F080E1ECE6F1E0A0E9B1E001900D924F
:102AF0008A95E1F781E001C080E01092260260969D
:102B0000EEE00C948A23783048F4693038F484304D
:102B100028F4462F672F0E94BB1C089580E090E0A8
:102B200008951F93CF93DF930E94D713EC01C11533
:102B300080E5D807E8F5C11590E4D90708F0A8C0EA
:102B4000C03ED10530F5CD3CD10508F094C0C83A5F
:102B5000D10578F4C53AD10508F083C0C130D1055C
:102B600009F47CC008F4F2C0C430D10508F0F1C00B
:102B7000EDC0C33CD10508F0E9C0C85AD0E0CC0F85
:102B8000DD1FCE5CDE4F0990D881C02DCE0194644C
:102B9000E1C0C11580E2D80708F0CBC0C11591E0B3
:102BA000D90708F06BC0C83ED10508F4D2C0CEC02A
:102BB000C03682E5D80728F5C03492E5D90708F079
:102BC00079C0C03282E5D80708F06CC0C11592E523
:102BD000D90708F481C04C2F4695469580E2489F5E
:102BE000A0011124C37021E030E0C90102C0880FA8
:102BF000991FCA95E2F7EA01C82BD92BCE019D682F
:102C0000A9C0C03A82E5D807B8F48C2F8F71C038BC
:102C100092E5D90708F07BC08695869590E2899F5A
:102C200090011124C37081E090E002C0880F991FC9
:102C3000CA95E2F79A6868C0C03C82E5D80708F4F4
:102C40006DC0C03E92E5D90708F080C0CF71DD2786
:102C5000DC2FCC27CE01806F906A7CC081E090E0B1
:102C600079C0C55AD0E0C15DDE4F8881C82FD0E061
:102C7000CE0190646FC0CE0190656CC08D2F0E9414
:102C80008813182FCE0199270E94D7131F715CC09B
:102C9000CE0199270E94D713CC27DF70D06A8C2BE6
:102CA0009D2B58C0CF71D0E0DC2FCC27CE01816F97
:102CB000906A50C08C2F8F718695869590E2899F7F
:102CC00090011124C37081E090E002C0880F991F29
:102CD000CA95E2F79C6818C08C2F8F710E948813E8
:102CE00095E0D695C7959A95E1F7CF70D0E0DC2FA7
:102CF000CC27282F30E084FF05C084E0220F331F4B
:102D00008A95E1F7D069CE01822B932B23C090E006
:102D1000D82FCC27CE01846F906A1CC08C2F8F7166
:102D20000E9488138F7190E0D82FCC27CE0190623B
:102D300011C08D2F8F710E948813182FCE019927F3
:102D40000E94D7131F719062912B04C080E090E025
:102D500001C0CE01DF91CF911F910895A6E0B0E0B0
:102D6000E4EBF6E10C9478230E94131A8C01809115
:102D70002202909123020817190781F019821A8202
:102D80000E94131A682F49815A81792F80E090E0C0
:102D90000E94DC2010932302009322022696E4E096
:102DA0000C94942380959091210289238093210291
:102DB000089580910C01813051F58091690287FF5F
:102DC00026C00E9473148093300240E250E069EF05
:102DD00071E08FE292E00E94A123892BD9F180E279
:102DE000EFE2F2E0A9EFB1E001900D928A95E1F7F0
:102DF000E0916502F0916602309761F186E0809380
:102E00002F020480F581E02D8FE292E022C00E9423
:102E100073148093270248E050E069E172E087E292
:102E200092E00E94A123892BA9F088E0E7E2F2E07A
:102E3000A9E1B2E001900D928A95E1F7E091650277
:102E4000F0916602309731F00280F381E02D87E245
:102E500092E0099508959091F601809589238093D9
:102E6000F601282F277069F4981759F090916A029B
:102E700092FF07C08695869586950E94351E109212
:102E8000F601089590916A0292FB222720F92817F3
:102E900079F080FB92F990936A02609169027091D7
:102EA0006A0284E090E00E94D32282E00E942B1705
:102EB00008958091F5019091BC01891719F08F5FF9
:102EC0008770FBCF0895CF93DF938091BB018295EC
:102ED0008F7009F04EC08091BA01882309F449C06F
:102EE0008091F5014091BC015091B6016091B5010E
:102EF000C091B701D091B80177E08417D1F190E08B
:102F0000789FF001799FF00D1124DF01A354BE4F8B
:102F100014962C911497222349F111962C91119714
:102F2000251324C02C91261321C015962C9115979A
:102F300021111CC012962D913C9113972C1B3D0B17
:102F4000283C310598F48091BB018F70806180939B
:102F5000BB01ED53FE4F80818F708061808385EBD4
:102F600091E00E945A030E94591703C0019687708E
:102F7000C4CFDF91CF910895A4E1B0E0E2ECF7E196
:102F80000C9470238C0186E0F801DE011F960190FD
:102F90000D928A95E1F7F8018481E58095EB892E01
:102FA00091E0992E9091B901911120C0882309F4E4
:102FB00063C1EE2009F442C0C8010E94511EF82EE0
:102FC0008823E1F187E0F801D40101900D928A9500
:102FD000E1F78091B901813031F48091B501909190
:102FE000B6010E94BC1D0E94631748C1F801D08041
:102FF000C180A280B380F090BA012091B7013091D6
:10300000B801FF2009F4E7C0A501421B530B483C5F
:10301000510508F09DC0882309F430C18091BB019F
:10302000282F207F9091B601222361F09C1509F48E
:1030300060C0C8010E94511E811163C0C8010E9476
:103040005A031AC19C1113C09091B5019D110FC074
:10305000E1100DC08F7080618093BB0185EB91E022
:103060000E945A038091BB01F801868303C1E110DD
:103070003AC040E06C2D8D2D0E94991440E06C2DDB
:103080008D2D0E949914E82E8111F4C0DF86C88A24
:103090008F8598890E94BC1D292F22952F7024307E
:1030A00020F49F70223028F009C02A50223080F08E
:1030B00014C0992349F0811107C013C0992321F04E
:1030C000F8019681907F69F0805E883030F409C005
:1030D000803F38F0815F833020F0C8010E945A039E
:1030E000EF2CFE2CCBC08091BB0181608093BB0193
:1030F000C1C09091B5019D119CCFE1109ACFF8010C
:1031000098C0EE2009F49ACF2091BB01822F8295BE
:103110008F7090E002978CF08091B5019091B6018C
:1031200099878887BB86AA868091B9018C871D867E
:103130002E87CE0108960E945A0387E0F801A5EB7E
:10314000B1E001900D928A95E1F70E94631794C057
:103150009091BB01292F207F51F485EB91E00E94D3
:103160005A0387E0F40111928A95E9F783C0882316
:1031700009F484C08091B6018C110CC08091B50116
:103180008D1108C0E11006C0F8019683C8010E94A5
:103190005A036AC0C8010E94511E882309F44ECF09
:1031A000EE2009F44BCF2091BB01822F82958F70C6
:1031B00090E0029714F28091B5019091B6019A8344
:1031C0008983BC82AB828091B9018D831E822F835B
:1031D000CE010196B0CFA21AB30AF8ECAF16B10433
:1031E00008F042C0882309F447C0FE2CEE2009F401
:1031F00025CF8091B6018C1129C08091B5018D1128
:1032000025C09091BB0190FD18C0892F82958F70C9
:10321000282F30E02115310581F0F80196832F30F9
:10322000310541F08F5F982F9295907F86818F7046
:10323000892B8683C8010E945A0387E0F801A5EB19
:10324000B1E001900D928A95E1F718C0C8010E9483
:10325000511E811172CF8091BB0181608093BB01AF
:10326000C8010E945A030AC087E0F40111928A95AE
:10327000E9F704C0F12C02C0FF24F3948F2D64966B
:10328000ECE00C948C2390917D0121E030E0F90179
:1032900001C0EE0F8A95EAF7D90102C0AA0FBB1F41
:1032A0006A95E2F7BD016E2B01C0220F4A95EAF73D
:1032B000892F8623681303C0892F822B03C0209592
:1032C000822F89230E94321E089580910B01089558
:1032D0000F931F93CF93DF938B01EA019091AB0182
:1032E000943079F58F708093E9008FEF9091E8002A
:1032F000815095FD06C095ED9A95F1F7000081117A
:10330000F5CF8091E80085FF1CC00E9453138823ED
:1033100061F08091E8008E778093E80012C0F80198
:1033200081918F018093F1002197209791F38091F3
:10333000E80085FDF4CF8091E8008E778093E80067
:10334000E4CFDF91CF911F910F91089540E250E0BB
:10335000BC0184E00E9468190895CF93DF93EC01CB
:1033600048E050E0BC0181E00E94681988E0FE015D
:10337000A1EAB1E001900D928A95E1F7DF91CF913A
:10338000089587E797E790930108809300089AE0F3
:1033900088E10FB6F894A895809360000FBE9093D3
:1033A0006000FFCF78941F920F920FB60F921124F6
:1033B0008F939F93AF93BF9380916C0290916D0216
:1033C000A0916E02B0916F020196A11DB11D809374
:1033D0006C0290936D02A0936E02B0936F02BF9146
:1033E000AF919F918F910F900FBE0F901F901895E6
:1033F0009C014FB7F89480916C0290916D02A0915E
:103400006E02B0916F024FBF821B930B08952FB7CE
:10341000F89460916C0270916D0280916E029091AF
:103420006F022FBF08952FB7F89480916C0290918E
:103430006D02A0916E02B0916F022FBF08951F928E
:103440000F920FB60F9211248F939F93AF93BF9358
:1034500080916B02811113C080916C0290916D027A
:10346000A0916E02B0916F024196A11DB11D809393
:103470006C0290936D02A0936E02B0936F02BF91A5
:10348000AF919F918F910F900FBE0F901F90189545
:1034900090910C01913021F49091690297FD03C045
:1034A000E7E2F2E01DC0E82FE695E695E695EE31FD
:1034B000E0F4F0E0E15DFD4F877021E030E0A9012C
:1034C00002C0440F551F8A95E2F7CA018095928188
:1034D000892382830895319652E0ED32F50729F071
:1034E00092818913F8CF1282F6CF089590910C0142
:1034F0009130D1F49091690297FF16C0E82FE695BC
:10350000E695E695EE3140F5F0E0E15DFD4F877020
:1035100021E030E0A90102C0440F551F8A95E2F76F
:10352000CA019281892B16C0A9E2B2E0EFEF90E0C8
:103530002D91821789F0EF3F19F4211101C0E92F75
:103540009F5F9630A9F7EF3F39F00E2E000CFF0B6E
:10355000E95DFD4F828308950895A3E0B0E0E3EBB9
:10356000FAE10C947A2320916702309168022817BF
:103570003907A1F09093680280936702E091650299
:10358000F0916602309751F024E029839B838A836F
:103590000084F185E02DCE01019609952396E2E0A5
:1035A0000C949623A3E0B0E0E8EDFAE10C947A23C2
:1035B000209163023091640228173907A1F090939B
:1035C000640280936302E0916502F0916602309795
:1035D00051F023E029839B838A830084F185E02DC9
:1035E000CE01019609952396E2E00C949623E09192
:1035F0006502F0916602309729F00190F081E02D8C
:103600000995089580E0089587E290E00E94B52230
:103610000895CF93C82F811102C06FEF01C065E2FA
:1036200084E290E00E94B522C11102C06FEF01C098
:1036300061E085E290E00E94B522C11102C06FEF07
:1036400001C064E186E290E00E94B522CF91089526
:1036500084E290E00E949722853281F485E290E036
:103660000E949722813051F486E290E00E949722D6
:1036700091E0843109F090E0892F01C080E08170F1
:1036800008950F931F93CF93DF93C42FD22FFC0184
:1036900085818823B1F0409362020E94131A9093AF
:1036A00061028093600280E28C0F883008F068C06D
:1036B000C77081E001C0880FCA95EAF70E94AC1E6E
:1036C0005FC08091620248133DC08091600290917A
:1036D00061020E94F819883C9105A0F510E21D0FC7
:1036E000CD17E9F080E28C0F883040F4C77081E09C
:1036F00001C0880FCA95EAF70E94A51E183078F518
:1037000081E09D2F977001C0880F9A95EAF70E947B
:10371000AC1E093351F560E570E089E329C0093337
:1037200019F460E570E002C060E070E0802F0E9454
:103730009F20183028F5D77081E001C0880FDA95F6
:10374000EAF70AC080E28C0F8830D0F4C77081E0BD
:1037500001C0880FCA95EAF70E94A51E11C009335F
:1037600051F460E570E089E309C060E070E0802F0B
:103770000E949F20E0CF60E070E0802F0E949F2099
:10378000DF91CF911F910F9108950E94131A2091FC
:103790005C02211104C020915D02222321F090934C
:1037A00059028093580220915E02211104C0209199
:1037B0005F02222321F09093570280935602E091FA
:1037C0006502F0916602309749F082E080935A02D8
:1037D0000680F781E02D8AE592E0099508958091B1
:1037E000550280FD16C081FD16C082FD18C0809173
:1037F0005402882391F0883290F428E0829FC0011F
:10380000112468E270E00E940D23862F672B29F0B7
:1038100007C082E0089584E0089581E0089588E07B
:1038200008958091550280FD14C081FD14C082FD71
:1038300016C080915302882381F08E3180F420E5F8
:10384000829FC00111246EE170E00E940D23862F3B
:10385000089584E1089588E2089588E0089580E558
:103860000895282F35EB2303C001112497FF03C0CF
:103870008058910902C080589F4F892F0895CF9397
:10388000DF93C8E6D2E060E0CE010E94B522219627
:10389000C11584E0D807B9F7DF91CF9108951F9340
:1038A000CF93DF93962F8430E8F46830D8F4493012
:1038B000C8F4632F122FC42FD0E0CC0FDD1F22E1FC
:1038C000929FC00DD11D112490E9899FC00DD11D7B
:1038D0001124CE0188960E94B522612FCE018996CF
:1038E0000E94B522DF91CF911F910895A0E0B0E032
:1038F000ECE7FCE10C947223A12CE12CF12CB12C0F
:1039000000E010E0C0E0D0E06701C00ED11EFE0173
:10391000EE0FFF1FEC0DFD1DEB5CFB4F259134916D
:103920004C2F6B2D8A2D0E944F1C2196C930D1053A
:1039300071F70E5E1F4FB39488E0B812E3CF80E9B1
:10394000E80EF11CA39484E0A812D9CFCDB7DEB75E
:10395000EAE00C948E2380E00E94091B60E070E096
:10396000CB010E94041B0E94761C0E943F1C81E038
:103970000E94091B08950F931F93CF93DF93843008
:1039800008F56830F8F44930E8F4C42FD0E0CC0FE3
:10399000DD1F22E1629FC00DD11D112430E9839FFC
:1039A000C00DD11D1124CE0188960E94972290E06F
:1039B000182F0027CE0189960E9497229801282B64
:1039C000C90102C080E090E0DF91CF911F910F917B
:1039D00008951F920F920FB60F9211242F933F93C9
:1039E0004F935F936F937F938F939F93AF93BF9307
:1039F000EF93FF9380910E0191E0980F823019F0C0
:103A000090930E014EC081E080930E01809151028F
:103A100090915202019660ED72E00E94F92290931B
:103A200052028093510265E070E00E94F92267FD26
:103A30006FE780915002823019F4603451F404C071
:103A4000813039F46F3729F480916F008E7F809335
:103A50006F00E62FF0E0EB54FC4F2491A09186001C
:103A6000B091870030E00E9450232FEF30E040E01B
:103A700050E00E942123C90163E070E00E94F92216
:103A800080914F02869586958695282F269FC001A6
:103A9000279F900D11240E9482219093890080938A
:103AA0008800FF91EF91BF91AF919F918F917F918E
:103AB0006F915F914F913F912F910F900FBE0F909B
:103AC0001F901895843030F4811105C090918000CA
:103AD0009F7704C083E0909180009068909380006D
:103AE000A0918600B0918700282F30E00E945023DB
:103AF00023E030E040E050E00E942123B42FA32FC8
:103B0000922F8827892F9A2FAB2FBB270E948221C3
:103B100090938900809388000895CF92DF92FF925E
:103B20000F931F93CF93DF936C0100917D018091E0
:103B30007C01082BC3E0D0E010E0C8010C2E02C0CD
:103B4000959587950A94E2F780FD04C02197A8F720
:103B5000F12C09C0FC2EB6018C2F0E9483150E9407
:103B60009115019799F38F2DDF91CF911F910F91AF
:103B7000FF90DF90CF900895CF93DF93EC010E94E8
:103B80008D1DBE010E9483150E949115DF91CF917A
:103B90000895292F983078F5893068F590E039E05C
:103BA000239F800D911D1124682F677023E0969547
:103BB00087952A95E1F7FC01EE0FFF1FE80FF91F2B
:103BC000E059FD4F40E050E080E0219130E0062ECA
:103BD00002C0369527950A94E2F721703327042E08
:103BE00001C0220F0A94EAF7822B4F5F5F4F4330E8
:103BF000510559F7089580E00895292F983088F5E8
:103C0000893078F590E039E0239F800D911D1124D3
:103C1000282F277051E001C0550F2A95EAF723E0BD
:103C2000969587952A95E1F7FC01EE0FFF1FE80FA7
:103C3000F91FE059FD4F20E030E070E04081CB01FA
:103C4000022E02C0969587950A94E2F781708195BD
:103C500084278523842781932F5F3F4F23303105AD
:103C600069F7089580937D01089521E030E001C057
:103C7000220F8A95EAF7209580917D0182230E9488
:103C8000321E089521E030E001C0220F8A95EAF744
:103C900080917D01822B0E94321E089580937C01C9
:103CA0000895FC0124812223D9F0808191810E9412
:103CB000BC1D92959F70963079F010F4925001C01F
:103CC0009A50923068F4803F69F018F4883E40F4CE
:103CD00009C0843F29F406C0883E20F0813F11F0DE
:103CE00080E0089581E008951092210280910C01F6
:103CF000813041F48091690287FF04C08EE1E1E3E5
:103D0000F2E003C086E0E9E2F2E0DF011D928A956D
:103D1000E9F780E090E00E94D21A80E090E00E94F3
:103D2000AD1A1092F8010E94D916EAE5F2E086E099
:103D3000DF011D928A95E9F7109253021092540206
:103D4000109255020E94C51B0895882321F00E94FD
:103D5000D2160E94D9160895882339F09091210235
:103D6000892B809321020E94D9160895662309F4B5
:103D70005CC08D3C21F40E94111C819504C08E3CD6
:103D800029F40E94111C80935D02C5C08F3C21F470
:103D90000E94111C819504C0803D29F40E94111CD1
:103DA00080935C02B8C0893D19F40E94EF1B05C0E6
:103DB0008A3D31F40E94EF1B819580935E02ABC077
:103DC0008B3D21F40E94EF1B819504C08C3D29F4AA
:103DD0000E94EF1B80935F029EC09FE2980F983075
:103DE00078F421E030E0A90102C0440F551F9A95F4
:103DF000E2F7CA0190915B02892B80935B028BC032
:103E00008D3D21F48091550281600CC08E3D21F4DE
:103E100080915502826006C08F3D09F07CC0809180
:103E2000550284608093550276C08D3C39F49091A0
:103E30005D0297FF35C010925D0259C08E3C29F497
:103E400090915D021916BCF32BC090915C028F3CDF
:103E500029F497FF25C010925C0249C0803D19F4F7
:103E60001916CCF31DC090915E02893D29F41916F4
:103E7000BCF410925E023BC08A3D19F497FF10C05B
